S113D000183C36C1FF2747C1002715C105272AC18F
S113D010042204C101242FBDD05A2000321838390B
S113D020C63FBDD0F8BDD0F8C60FBDD0F8C606BD0A
S113D030D0F8C601BDD0F820E3BDD106BDD0B418E8
S113D0403018A70020D6BDD0D6BDD0AB20CEE60088
S113D050C10427C8BDD05F0820F4C104260139C12A
S113D0600D2604BDD07139BDD0FFBDD106BDD07829
S113D07039BDD106BDD089398114272381402727A2
S113D0808154271F810027113981132312812723FB
S113D090168153230E8167230086018080200C862D
S113D0A040200886142004865420003716CB80BD07
S113D0B0D0F8333981132204C601201881272206AF
S113D0C0C6038014200E81532206C6028040200429
S113D0D0C60480544C398100270781142302860139
S113D0E04AC1012712C10226048B40200AC103262B
S113D0F0048B1420028B5439F72000BDD11439F766
S113D1003000BDD1143918CE0002B620002BFB1814
S110D1100926F73918CE0800180926FC3945
S105FFE6C057FE
S105FFDCC07BE4
S105FFFEC0003D
S113C0008E00FFCE10008640A7228620A72486102B
S113C01097006F260ECE10007F00016F271F264069
S113C020FC1E2640FCC600BDD0009601E627CE27A4
S113C03010BDC04ECE03E8BDC04ECE0064BDC04EA0
S113C040CE000ABDC04ECE0001BDC04E20C7028F37
S113C050CB30BDD0008F39CE10001F23401C86404A
S113C060A723EC18C3F424ED187A0000260C8620CC
S113C0709700A6268840A726A7043BCE10001F25BC
S10DC08020078620A7257C00013B61
S9030000FC
